:1000000000308A00272800001030840000080319FF
:10001000182801308D008C018C0B0C288D0B0B28BF
:100020004A308C008C0B122800000000800B09283D
:10003000003411308400FC308005800C800C0008F6
:100040000319262824280000800B2328003484016B
:100050001F308305831685148312851C7B28831625
:100060000512831205160130900004200230900022
:10007000EC3091001920900B38288316051283125A
:100080000512831685118312851501309000042016
:1000900002309000EC3091001920900B4A28831612
:1000A0008511831285118316051183120515013000
:1000B0009000042002309000EC3091001920900B49
:1000C0005C2883160511831205118316051083120F
:1000D000051401309000042002309000EC309100B3
:1000E0001920900B6E2883160510831205100A3014
:1000F000900004202A288316851483128518ED2881
:100100008F010F08633C031CB62883160512831267
:100110000516013090000420831605128312051283
:1001200083168511831285150130900004208316F3
:10013000851183128511831605118312051501306F
:1001400090000420831605118312051183160510F3
:1001500083120514013090000420831605108312C9
:1001600005100A30900004208F0A81288F010F08A3
:10017000633C031CEC28831605128312051602301B
:100180009000042083160512831205128316851130
:100190008312851502309000042083168511831286
:1001A0008511831605118312051502309000042075
:1001B0008316051183120511831605108312051489
:1001C00002309000042083160510831205100A30B7
:0E01D000900004208F0AB7287B282A2863009D
:02400E00F93F78
:00000001FF
